:104777000000770101010200000301FA0400FA05B5
:1047870000020A0A5A0B000F0C00FA0D00030E0074
:10479700030F0132100096120132130AFA140102B4
:1047A70015000017010A18010A1905321A010A1B18
:1047B700010A1C053223011E2400642A00FA2B007B
:1047C700FA2C50782D003C2E00462F001E30006436
:1047D7003250783300003432FA35016436016437D9
:1047E7000150380A643C00643E003C3FFFFF40FF35
:1047F700FF411450420A5A430AC84405324500781B
:104807004600FA47FFFF4802034C00FA4EFFFF50ED
:104817000606510596521432530B28540A96560130
:1048270002570546580002590A465A32FA5B010AEE
:104837005C14325E000A5F00FE61FFFF64FFFF67E2
:1048470001036A0A3C6B00006C32967801327901E9
:1048570032FAFAFA0000770101010200000301FAB7
:104867000400FA0500020A0A5A0B000F0C00FA0DA1
:1048770000030E00030F0132100096120132130AD3
:10488700FA14010215000017010A18010A19053266
:104897001A010A1B010A1C053223011E2400642A7F
:1048A70000FA2B00FA2C50782D003C2E00462F00E2
:1048B7001E3000643250783300003432FA35016418
:1048C700360164370150380A643C00643E003C3FBF
:1048D700FFFF40FFFF411450420A5A430AC84405EC
:1048E700324500784600FA47FFFF4802024C00FABB
:1048F7004EFFFF500606510596521432530B2854AB
:104907000A96560101570546580001590A465A3278
:10491700FA5B010A5C14325E000A5F00FE61FFFF6A
:1049270064FFFF6701036A0A3C6B00006C329678EC
:104937000132790132FAFAFA0065006F00790083D3
:10494700008D009700A100AC00B600C000CA00D4DB
:1049570000DE00E800F2005B0063006A0072007A84
:10496700008200890091009900A100A800B000B85A
:1049770000BF00C700CF00D600DF00E600EE00F65C
:1049870000400046004C00520059005F0065006B74
:1049970000710077007D00830089008F0095009CDF
:1049A70000A200A800AE00B400BA00C000C600CC48
:0C49B70000D200D900DF00E500EB00F1A9
:10009E00AE33AF3474788E048F05FF1200858C3525
:1000AE008D36AE33AF3474788E048F05FF124C4606
:1000BE008C338D34E534453360137478C39534FF37
:1000CE00E49533FE8E338F347835124C92229000A5
:1000DE0078E0B40104C20C8002D20C900079E0B436
:1000EE000104C20D8002D20D9000B6E075F06EA430
:1000FE00FFAEF0740A8E048F05FF12008590079EE6
:10010E00ECF0A3EDF0A208401674038C068D0712D6
:10011E004C2B7401124C1D90079CEEF0A3EFF07E59
:10012E00017F00900074E0124C2B9000B7E08E041B
:10013E008F05FF120085740AFF1200858D3990001D
:10014E00C0E075F06EA4FFAEF0740A8E048F05FF4A
:10015E001200859007A2ECF0A3EDF09000C2E060D3
:10016E00139000C2E0F5F0741684FF7E00EF900746
:10017E00AAF0800674649007AAF09000A1E0B40B78
:10018E000874E3900063F080499000A1E0B4191266
:10019E009000B7E090492A124C0EE493900063F061
:1001AE0080309000A1E0B41E129000B7E090494854
:1001BE00124C0EE493900063F080179000A1E0B40F
:1001CE0028109000B7E0904972124C0EE493900004
:1001DE0063F09000BCE0B4020674029000ACF090A4
:1001EE00003FE0C39405502274019000BAF09000D5
:1001FE00BCE0B4020674019000BCF09000ACE0D3F9
:10020E009402400674029000ACF09000D4E0B40169
:10021E0017900024740FF0A374FFF0900026E4F002
:10022E00A3F074029000D4F09000D4E0B403419097
:10023E000026E0FEA3E0FF900024E0FCA3E0FD1208
:10024E004C8A7410124C2B7408124C1DEF900060E7
:10025E00F0EF700674FF900060F074009000D4F020
:10026E00900025E0900061F0900024E0900062F094
:10027E009000307401F07402900031F0740390001D
:10028E0032F022C293C294C291C292C287C290E54A
:10029E00B554EFF5B5E5B554DFF5B5C296C295C2C6
:1002AE00A0C297C2A2C2A1E5B5547FF5B5E5B5547B
:1002BE00BFF5B5E5B554FBF5B5C20E7537469000E2
:1002CE00AEE07005754902800375490390000C7409
:1002DE00FFF0A374DCF090008FE0900012F8E4F0D1
:1002EE00E8A3F0C214C216C21874C890002AF074A3
:1002FE00C890002CF074C890002EF075260075255D
:10030E0000C208756C00E54BB40903754B00753CD3
:10031E000090001AE4F0A3F0754C1E7528007527A6
:10032E0000C211C212C21390079EE0FEA3E0FF743A
:10033E0003124C2B7401124C1D90079CEEF0A3EF90
:10034E00F0C203900010E4F0A3F0C21F22053D227C
:10035E0085A74F75A7109000ACE0B4032CA2D8B3BC
:10036E004002C293A2D9B34002C294A2DAB34002B1
:10037E00C291A2DBB34002C292A2DCB34002C2879A
:10038E00A2DDB34002C290801BA2D8B34004C29338
:10039E00C292A2D9B34004C294C287A2DAB3400477
:1003AE00C291C29075D840854FA722900047E49322
:1003BE006406600280FE74C89007A4F8E4F0E8A317
:1003CE00F075B50075840175A70075FF8075EF0691
:1003DE00900033E4F075C91075A70F75A1C775A706
:1003EE000075D90075CE0C75A70F75F1FE75F2FF6D
:1003FE0075F30775F47875A4BA75A5FF75A607751C
:10040E00AE0075AFFF75D48175D5FF75D6FF75D764
:10041E00FF75A70075A20175A14775F80975D8007B
:10042E0075D90475A71075D80075D90475DA0975D4
:10043E00DB0975DC0975DD0975DE0975DF0975D80F
:10044E004075A70075E60075E71075BC0175BE0412
:10045E0075BD6C75BE0775BDA075BE0875BD017501
:10046E00BC0075BB1875BC2075BA0875E88075D1CF
:10047E001375B50075A70F75E10575E20075C740D8
:10048E00C293C294C291C292C287C290E5B554EF94
:10049E00F5B5E5B554DFF5B5C296C295C2A0C297C3
:1004AE00C2A2C2A1E5B5547FF5B5E5B554BFF5B509
:1004BE00E5B554FBF5B5759700759780740A120073
:1004CE00757597C0E5975420700280F8758F027588
:1004DE00A700D2AF75980075A90C75A70F75AB4321
:1004EE0075ADFB75AC1E75A71075C91875CA00756C
:1004FE00CB0075C80475A700758912758E04758CAE
:10050E0000758A00C2A9D28C758D00758B00D2AB96
:10051E00D28E75D944753200753100752E00752D49
:10052E0000754600754700C2997509C87508001216
:10053E002BCD75B50074639007A4F8E4F0E8A3F032
:10054E00122E59750964750800122BCDC21E90002B
:10055E004EE0B40108A2B54002D21E802E90004E8D
:10056E00E0B4021175A70F75F30F75A700A2A34093
:10057E0002D21E801690004EE0B4030F75A70F75C1
:10058E00F31775A700A2A44002D21EA21EB35003F9
:10059E0002068074089007A4F8E4F0E8A3F0122D88
:1005AE0028750964750800122BCD74099007A4F8FC
:1005BE00E4F0E8A3F0122D28750964750800122BDB
:1005CE00CD740A9007A4F8E4F0E8A3F0122D287574
:1005DE000964750800122BCD740B9007A4F8E4F093
:1005EE00E8A3F0122D28750964750800122BCD743E
:1005FE000C9007A4F8E4F0E8A3F0122D2875096416
:10060E00750800122BCD740D9007A4F8E4F0E8A342
:10061E00F0122D28750964750800122BCD740E90FA
:10062E0007A4F8E4F0E8A3F0122D28750964750804
:10063E0000122BCD74029000ADF090004EE09000B1
:10064E0071F090004EE0B401087400900079F080D3
:10065E001C90004EE0B4020874009000BCF0800DB7
:10066E0090004EE0B4030674009000C9F0D21B0255
:10067E0007599007A4E4F0A304F0122D287509641D
:10068E00750800122BCD74029007A4F8E4F0E8A3CD
:10069E00F0122D28750964750800122BCD74039085
:1006AE0007A4F8E4F0E8A3F0122D28750964750884
:1006BE0000122BCD74049007A4F8E4F0E8A3F01216
:1006CE002D28750964750800122BCD74059007A4AA
:1006DE00F8E4F0E8A3F0122D2875096475080012ED
:1006EE002BCD74069007A4F8E4F0E8A3F0122D28A1
:1006FE00750964750800122BCD74079007A4F8E4F1
:10070E00F0E8A3F0122D28750964750800122BCDA0
:10071E0074019000ADF090004EE0900071F09000EA
:10072E004EE0B401087400900079F0801C90004EE9
:10073E00E0B4020874009000BCF0800D90004EE012
:10074E00B4030674009000C9F0C21B122FCD9000A6
:10075E00B7E07006740A9000B7F0900063E0700680
:10076E0074E3900063F01200DCE5B54401F5B57456
:10077E000690003DF0740190003EF074039000402E
:10078E00F07404900041F07428900042F0740590CB
:10079E000043F090003FE0B404067404900043F070
:1007AE007403900044F07400900049F074009000BF
:1007BE004AF0740190004BF0740090004CF074FFFE
:1007CE0090004DF0744E90013BF0746990013CF036
:1007DE00747390013DF0747390013EF0746190015A
:1007EE003FF0746E900140F07420900141F0743629
:1007FE00900142F07443900143F07479900144F0FB
:10080E00746C900145F07420900146F074209001B4
:10081E0047F07420900148F07420900149F0900048
:10082E00D3E0900060F090008AE0900061F09000BC
:10083E008BE0900062F0C214C216C21874C8900009
:10084E002AF074C890002CF074C890002EF0C211DB
:10085E00C212C213A2B6B3920AA2B3B3920BC209CA
:10086E00752600752500753746754C1E90005CE4A4
:10087E00F075271975286490000C74FFF0A374DCD2
:10088E00F0C20E754B00C208752A00752900900043
:10089E0010E4F0A3F0743A900764F074FD900765CD
:1008AE00F0756D0090005DE4F0752C00752B0090D6
:1008BE0000287475F0A37430F0900014E4F0A3F0E7
:1008CE0090008FE0900012F8E4F0E8A3F090007032
:1008DE00E075F032A4FFAEF0900022EEF0A3EFF040
:1008EE0090079EE0FEA3E0FF7403124C2B740112DE
:1008FE004C1D90079CEEF0A3EFF0754A0174FA9030
:10090E000039F0C21F756C00753C00C20FC210C2D8
:10091E0020C203754D00C204D205C206D207C21C06
:10092E00C21D74FE900034F074FE900035F07538E0
:10093E0000754400753A00753E32753F00754000F3
:10094E00743C900037F0743C900038F0754100759F
:10095E00420075430090001AE4F0A3F0754500D2F2
:10096E00B2D2A4D2B0D2B1D2A3D2A7D2A6D2A5D29D
:10097E00B7900070E0D394FA400674FA900070F0CD
:10098E007E017F00900062E0124C2B900061E02F00
:10099E00FF50010E900024EEF0A3EFF0EFD394FF82
:1009AE00EE940F4007900024E4F0A3F0900060E076
:1009BE00700674FF900060F09000ADE0D39402409A
:1009CE000674019000ADF09000AEE070057549021E
:1009DE0080037549039000AFE0D394014006740084
:1009EE009000AFF09000B5E0C3940A5006740A90E0
:1009FE0000B5F09000BFE0700674019000BFF0905B
:100A0E0000BFE0B4FF0674FE9000BFF09000C6E099
:100A1E00D394FE400674FE9000C6F074019000CC94
:100A2E00F074019000CDF074009000CFF07400903F
:100A3E0000D4F0D29CD2EC75CF01A298B350030231
:100A4E000E35C298E54764046006E59964FF6002BE
:100A5E00801EE547600874E62547900039F075471B
:100A6E0000E546600874F02546900039F0754600A2
:100A7E00E5476003020B20754700E599B4FF037547
:100A8E004601E599B4FE03754602E599B4FD03757A
:100A9E004603E599B4FC03754604E599B4FA03756B
:100AAE004605E599B4FB03754701E599B4F903755D
:100ABE004704E599D394E54007E599C394F04002C5
:100ACE0080168599487547027E017F00E548C394DC
:100ADE00E6124C2B8E2F8F30753200753100E59952
:100AEE00D394C74007E599C394E64002801F8599C9
:100AFE004875470374E5C39548F530752F00AE2F42
:100B0E00AF309049C31200647831124C70D2990202
:100B1E000E35E547B401028003020BFCE532453188
:100B2E007003120291AE31AF32900064124C52E556
:100B3E0099F07831124C92AE31AF32EFB40106EE2D
:100B4E00B407028003020BFC900764E0B43C028001
:100B5E0003020BE6C29C1200DC900060E09000D312
:100B6E00F0900061E090008AF0900062E090008BBF
:100B7E00F0A21B4031755001E550D394075025E586
:100B8E00509007A4F8E4F0E8A3F074AA900033F0B4
:100B9E00122BF9750964750800122BCD785074016B
:100BAE0026F650D4802F755008E550D3940E50255C
:100BBE00E5509007A4F8E4F0E8A3F074AA9000338F
:100BCE00F0122BF9750964750800122BCD7850744C
:100BDE000126F650D4122FCD74C89007A4F8E4F075
:100BEE00E8A3F0D29C7547007546007599FBE54762
:100BFE00B402028003020C90E532453170068599ED
:100C0E002E752D00AE31AF3274016F4E701BAC2DB0
:100C1E00AD2EAA2FAB30ED2BFBEC3AFA8A068B07E2
:100C2E00900064124C52E599F07831124C92AE312C
:100C3E00AF3274026F4E704AAC2DAD2E740D6D4CEA
:100C4E00702774639007A4F8E4F0E8A3F074AB90F7
:100C5E000033F0900071E090004EF0122F3274C805
:100C6E009007A4F8E4F0E8A3F0AE2DAF2E74566F03
:100C7E004E70031202911200DC854899754700757B
:100C8E004600E547B4033FAE31AF32900064124CDC
:100C9E0052E599F07831124C92AE31AF32AC2FADA5
:100CAE00308F028E038C068D079049FF120064E48C
:100CBE0093F9740193FEEAD39EEB99400985489906
:100CCE00754700754600E547B404028003020E35F1
:100CDE00E53245317003120291AE31AF32900064AD
:100CEE00124C52E599F07831124C92AE31AF32EF90
:100CFE00B40006EEB401028003020E35900047E008
:100D0E0075F002A4FDACF08D50ED900064124C67AE
:100D1E00EDFAE0FBEA900067124C67EBFAE0FBEAB3
:100D2E002BFA900047E0B502028003020E270DED6C
:100D3E00900064124C67E550FDE0FAED90006812E9
:100D4E004C67EAFDE0FAEDC39AFD900047E0B50569
:100D5E00028003020E27E550900066124C67E550A4
:100D6E00FDE0FAED900069124C67EAFDE0FAED2A1B
:100D7E00FD900047E0B505028003020E27E5509076
:100D8E00006A124C67FDE0FAED900047E0F4042A89
:100D9E0090004EF0E55090006B124C67FDE0FAEDBE
:100DAE00900047E0F4042A90004FF0E55090006C5C
:100DBE00124C67FDE0FAED900047E0F4042A900033
:100DCE0050F0E55090006D124C67FDE0FAED90008A
:100DDE0047E0F4042A9007A4F8E4F0E8A3F074AB1B
:100DEE00900033F0122F32750964750800122BCD66
:100DFE009007A4124C39122F32750964750800122F
:100E0E002BCD9007A4124C39122F327599F9750912
:100E1E0064750800122BCD80FE7599FF75096475F7
:100E2E000800122BCD80FEE5466006A299B3B340B2
:100E3E0003020FB3C299E546B4011FAE31AF329033
:100E4E00003D124C52E0F5997831124C92AE31AF12
:100E5E003274116F4E7003754600E546B402038579
:100E6E004A99E546B4031DAE31AF32900064124C80
:100E7E0052E0F599EFB40107EEB40703754600781A
:100E8E0031124C92E546B404028003020F75E5322E
:100E9E0045317003852699AE31AF3274016F4E70B5
:100EAE0003853899AE31AF3274026F4E7003853AB6
:100EBE0099AE31AF3274036F4E7003853E99AE31E9
:100ECE00AF3274046F4E7003854099AE31AF3274F9
:100EDE00056F4E7003854199AE31AF3274066F4E79
:100EEE007003854299AE31AF3274076F4E70038531
:100EFE004399AE31AF3274086F4E700690001BE00E
:100F0E00F599AE31AF3274096F4E7006900039E02C
:100F1E00F599AE31AF32740A6F4E7003854499AEB7
:100F2E0031AF32740B6F4E7003853F99AE31AF32D5
:100F3E00740C6F4E7003854599AE31AF32740D6FE0
:100F4E004E7005900039E4F0AE31AF32740D6F4E35
:100F5E0070037599FC7831124C92AE31AF32740E2B
:100F6E006F4E7003754600E546B4053990003FE0BC
:100F7E00D394044010AE31AF32904777124C52E406
:100F8E0093F599800EAE31AF3290485B124C52E41D
:100F9E0093F599AE31AF3274E36F4E700375460020
:100FAE007831124C92E54764016005E547B40403BD
:100FBE00020A45C28E7E087F00E53D124C2BE58D60
:100FCE0075F008A4FDACF0EF2DFDEE3CFCE58B7545
:100FDE00F02084FF7E00ED2FFFEC3EFE8E278F2843
:100FEE00D28E900091E0605690001C124C39900009
:100FFE001CE0FCA3E0FD90001EE0FAA3E0FBEDB5C3
:10100E00033CECB50238B21AA208B34013A21AB3CD
:10101E004008E5B54404F5B58006E5B554FBF5B5D5
:10102E0090001EE0FEA3E0FF900020E0FCA3E0FD98
:10103E00EF2DFDEE3CFC90001EECF0A3EDF09000C9
:10104E009EE0600990009EE0C3940340030210E10D
:10105E001244CDA208B3500990005CE0C3940D4039
:10106E00028006900088E0F56BE56B75F005A4FF35
:10107E00AEF09007A6EEF0A3EFF0900075E0C395EA
:10108E003A4007E538C3953950079007A6E4F0A318
:10109E00F0AE58AF599007A6E0FCA3E0FDEFD39D4C
:1010AE00EE9C4004C2A1800B90005CE0C3941450EF
:1010BE0002D2A190009EE0B402129000ACE0C39464
:1010CE000350099000BCE0C3940240028005A2A127
:1010DE00B392A290009EE0B4031C1245C9AE58AF65
:1010EE00599007A6E0FCA3E0FDEFD39DEE9C4004D3
:1010FE00D2A18002C2A1A2B6300A01B350030215DA
:10110E0078A2B6300A01B35003021578A2B6300C9D
:10111E0001B3500302147E754A00900091E07013E3
:10112E00A20CB34008E5B554FBF5B58006E5B54411
:10113E0004F5B50537A209B3407DE549B40330E5A2
:10114E0037B40705754901801FA21FB3401AE53752
:10115E00C3940750069000397401F0E537D3940715
:10116E0040067402900039F0753701D21F8044E5B5
:10117E0049B40206754901753704E537B40405759F
:10118E003701802F900039E0701AE537C394045070
:10119E00069000397401F0E537D3940440067402CA
:1011AE00900039F09000AEE0B40205120291800377
:1011BE00753701C209D21DE549C394035006E537C0
:1011CE00640460028005753701C21DE537B403491A
:1011DE00900091E0604390001CE0FEA3E0FF9000C1
:1011EE0091E08E048F05FF12008574018C068D0729
:1011FE00124C1D900020EEF0A3EFF0900020E0F8CE
:10120E00A3E090001EC8F0A3C8F090001CE4F0A369
:10121E00F0C21AE5B554FBF5B5AE2BAF2CAC27AD2D
:10122E0028EF2DFDEE3CFC8C2B8D2CAE27AF28EF3E
:10123E00D39DEE9C4011900014E0FAA3E0FBEBC3AB
:10124E0094E8EA940340028006900014124C399000
:10125E00000CE527F0A3E528F090000EE527F0A39B
:10126E00E528F0AE27AF28740C8E048F05FF120010
:10127E00858C298D2AC28E758D00758B00753D006B
:10128E00752801752700D28E90000CE0FEA3E0FFBA
:10129E00EF4E600B7C587DF9124B2D8E258F26AEAE
:1012AE0025AF267428BE00039F5010E53C2FFF503B
:1012BE00010E7401124C1D8E258F2685263C75CD90
:1012CE000075CC00753D009000B5E0A825B8000D66
:1012DE00D395264008E526900036F080099000B59B
:1012EE00E014900036F0E54960067526007525007D
:1012FE00E53764016005E537B4030312420FE54B91
:10130E00B40903754B00A20F500302140590006A36
:10131E00E0B4015AE54075F00584FF7E0090056447
:10132E00124C52E0F534753300AE33AF3490006892
:10133E00E0124C2B74648E048F05FF12008574C16D
:10134E008C068D07124C2B8E358F36900012E0FED8
:10135E00A3E0FFAC33AD3412000374648E048F052A
:10136E00FF120085900012ECF0A3EDF0800F9000BC
:10137E0068E075F0C1A4FFAEF08E358F36E53AC346
:10138E0094CC507175A71085F95085FA517E017F66
:10139E0000E551124C2BE5502FFF50010E8E338F6E
:1013AE0034AC35AD36EF2DFDEE3CFC8C358D36D2A2
:1013BE0093D294D291E536F5FBE535F5FCE536F59D
:1013CE00E9E535F5EAE536F5EBE535F5EC9000ACFB
:1013DE00E0B4031ED292D287D290E536F5EDE53514
:1013EE00F5EEE536F5FDE535F5FEE536F5CEE535FA
:1013FE00F5CF75A700D20FE549B4010F754C0190DA
:10140E00003C7401F0E5B54401F5B5E549705C901A
:10141E0000B1E0600D9000B8E0A825B80006952652
:10142E00400280239000B1E0B40208754C0375456C
:10143E0000800CC20075450090001AE4F0A3F07411
:10144E0009900039F08024754C01E537B4010690FF
:10145E00003C7401F0E537B40206740290003CF0D3
:10146E00E537B40306740390003CF0A20CB3920A65
:10147E00A20CB330B601B35003021578754A01A21F
:10148E000C920AE537D394484012D20EE537D39426
:10149E004E40097403900039F07537469000B9E05C
:1014AE00B40107E543C39414400280031202917401
:1014BE000D90005CF0A20EB3B35018900028E0FE21
:1014CE00A3E0FF7402124C2BAC27AD28EFC39DEEA8
:1014DE009C40028002D209900028E527F0A3E5285F
:1014EE00F0A204300501B35017A204B34008E5B5CD
:1014FE004408F5B58006E5B554F7F5B5A204920596
:10150E00A206300701B35017A206B34008E5B54452
:10151E0002F5B58006E5B554FDF5B5A2069207E5D0
:10152E0043C394415009740E900039F01202919009
:10153E000043E0FE90003FE004C39E400990003F50
:10154E00E0D39406400974FB900039F0120291909A
:10155E000048E06015900048E0FE900042E06E60AA
:10156E000974FE900039F0120291A211B3B3500625
:10157E00E53764026003021656A202B35006A200BB
:10158E00B3B3400302165075A71085F95085FA5172
:10159E007E017F00E551124C2BE5502FFF50010EBE
:1015AE008E338F34900018E0FCA3E0FDEF2DFDEE9E
:1015BE003CFC8C358D369000ACE0B4034EA208B3E3
:1015CE004028A21DB3400CE536F5FBE535F5FCD2FF
:1015DE0093800AE536F5EDE535F5EED292A203B32A
:1015EE004004D2978002C297801FE536F5FBE535A1
:1015FE00F5FCE536F5EDE535F5EED293D292A20384
:10160E00B34004D2978002C2978011E536F5FBE510
:10161E0035F5FCD293A203B34002D2929000CAE0F9
:10162E00B4021CAE33AF34AC56AD57EF2DFDEE3CCD
:10163E00FC8C358D36E536F5EBE535F5ECD292754D
:10164E00A700C211D212D213A212B3B35006E537BD
:10165E0064036003021734A202B35006A200B3B3B0
:10166E00400302172E75A71085F95085FA517E0199
:10167E007F00E551124C2BE5502FFF50010E8E339B
:10168E008F34900018E0FCA3E0FDEF2DFDEE3CFC46
:10169E008C358D369000ACE0B4034EA208B34028D2
:1016AE00A21DB3400CE536F5E9E535F5EAD2948096
:1016BE000AE536F5FDE535F5FED287A203B3400403
:1016CE00D2978002C297801FE536F5E9E535F5EA37
:1016DE00E536F5FDE535F5FED294D287A203B3408B
:1016EE0004D2978002C2978011E536F5E9E535F50B
:1016FE00EAD294A203B34002D2879000CAE0B402A9
:10170E001CAE33AF34AC56AD57EF2DFDEE3CFC8C1A
:10171E00358D36E536F5FDE535F5FED28775A70034
:10172E00D211C212D213A213B3B35006E53764011D
:10173E006003021812A202B35006A200B3B3400314
:10174E0002180C75A71085F95085FA517E017F009D
:10175E00E551124C2BE5502FFF50010E8E338F3476
:10176E00900018E0FCA3E0FDEF2DFDEE3CFC8C3567
:10177E008D369000ACE0B4034EA208B34028A21DF3
:10178E00B3400CE536F5EBE535F5ECD291800AE584
:10179E0036F5CEE535F5CFD290A203B34004D297FD
:1017AE008002C297801FE536F5EBE535F5ECE536A0
:1017BE00F5CEE535F5CFD291D290A203B34004D247
:1017CE00978002C2978011E536F5EBE535F5ECD240
:1017DE0091A203B34002D2909000CAE0B4021CAEB4
:1017EE0033AF34AC56AD57EF2DFDEE3CFC8C358D42
:1017FE0036E536F5CEE535F5CFD29075A700D21188
:10180E00D212C213E54CB40818123B3EA211B350CB
:10181E0005A212B340028006D211D212D213754C19
:10182E001EE54CB407061238F6754C08E54CB406A6
:10183E003D900012E0FEA3E0FFEF4E6006A208B35B
:10184E00B340028023AE52AF53900012E0FCA3E0EF
:10185E00FDEF2DFDEE3CFC8C528D53E537D39401FC
:10186E0050069000121200391236C8754C07E54C1E
:10187E00B40506123528754C06E54CB404329000BA
:10188E009FE0902BAFF82828731231BC80121231D2
:10189E00BC800D12336A800812341C800312341C73
:0F2BAF0002189702189C0218A10218A60218AB70
:1018AE00900081E060051242F88002C204754C057A
:1018BE00E54CB4030280030219A8900084E0600591
:1018CE001243E88002C20690009FE0D39402403F8C
:1018DE00900073E02403A825B800049526500990C3
:1018EE000075E0D3953A50028008D2027408900039
:1018FE0039F0900073E0A825B80005D39526500B5B
:10190E00900075E02403C3953A5002C202803990CC
:10191E000073E02403A825B8000495265007E53887
:10192E00C3953940028008D2027408900039F090B5
:10193E000073E0A825B80005D395265009E5392493
:10194E000FC395385002C2029000B9E07007E5430C
:10195E00C3941440028002D202A2024005754C04C8
:10196E00800A754C1E90001AE4F0A3F0A208B34052
:10197E0029E54075F00584FF7E00900564124C52F7
:10198E00E0C394695005124244800F90079EE0F820
:10199E00A3E090079CC8F0A3C8F0E54CB40A0280FF
:1019AE0003021A7890002BE0C394465008C2967436
:1019BE004690002BF0855A34753300900030E0F5D8
:1019CE005012009EE53690002BF0900006E533F0A5
:1019DE00A3E534F0C215900065E0FE90002BE0C345
:1019EE009E5012900065E0FE90002BE0F4042E90C5
:1019FE00002BF08012900065E02403FE90002BE097
:101A0E00F4042E90002BF09007A0E0F533A3E0F540
:101A1E0034900030E0F55012009EE53690002AF02A
:101A2E00900000E533F0A3E534F0C214900065E0B9
:101A3E00FE90002AE0C39E5012900065E0FE9000DA
:101A4E002AE0F4042E90002AF08012900065E02423
:101A5E0003FE90002AE0F4042E90002AF0E549B42B
:101A6E000105754C0B8003754C0390002AE0B537C9
:101A7E00028003021B10A214406B900000E0FEA334
:101A8E00E0FFEF4E605DAC25AD26740ABC0033D38B
:101A9E009D402FAA29AB2A74058A048B05FF1200DC
:101AAE00858D068C07900000E0FCA3E0FDCFCECF25
:101ABE001200037401124C1D900000EEF0A3EFF023
:101ACE008021AE29AF2A900000E0FCA3E0FD1200B9
:101ADE0003740A8E048F05FF120085900000ECF04F
:101AEE00A3EDF0D214AE27AF28900000E0FCA3E0E7
:101AFE00FDEFC39DEE9C400AD296C21474C89000AE
:101B0E002AF0A214B3B3500790002AE0B537028032
:101B1E000AD29674C890002AF0C21490002BE0B539
:101B2E0037028003021BC1A215406B900006E0FE37
:101B3E00A3E0FFEF4E605DAC25AD26740ABC00330A
:101B4E00D39D402FAA29AB2A74058A048B05FF1258
:101B5E0000858D068C07900006E0FCA3E0FDCFCE3D
:101B6E00CF1200037401124C1D900006EEF0A3EF8D
:101B7E00F08021AE29AF2A900006E0FCA3E0FD1212
:101B8E000003740A8E048F05FF120085900006EC88
:101B9E00F0A3EDF0D215AE27AF28900006E0FCA31F
:101BAE00E0FDEFC39DEE9C400AC296744690002B5A
:101BBE00F0C215A215B3B3500790002BE0B5370253
:101BCE00800AC296744690002BF0C215E54CB40BF9
:101BDE00028003021CCB90002DE0C394465013905C
:101BEE0000BAE0B40104C2968002C2957446900019
:101BFE002DF0855A34753300900031E0F550120007
:101C0E009EE53690002DF0900008E533F0A3E53404
:101C1E00F0C217900065E004FE90002DE0C39E50C8
:101C2E0013900065E004FE90002DE0F4042E900069
:101C3E002DF08012900065E02404FE90002DE0F45B
:101C4E00042E90002DF09007A0E0F533A3E0F534BC
:101C5E00900031E0F55012009EE53690002CF09089
:101C6E000002E533F0A3E534F0C216900065E004FF
:101C7E00FE90002CE0C39E5013900065E004FE9091
:101C8E00002CE0F4042E90002CF08012900065E001
:101C9E002404FE90002CE0F4042E90002CF0E54974
:101CAE00B4011774C890002AF074C890002CF07418
:101CBE00C890002EF0754C0C8003754C0390002CD0
:101CCE00E0B537028003021D6EA216406B90000233
:101CDE00E0FEA3E0FFEF4E605DAC25AD26740ABCBE
:101CEE000033D39D402FAA29AB2A74058A048B0595
:101CFE00FF1200858D068C07900002E0FCA3E0FD2C
:101D0E00CFCECF1200037401124C1D900002EEF0E4
:101D1E00A3EFF08021AE29AF2A900002E0FCA3E0F1
:101D2E00FD120003740A8E048F05FF1200859000C9
:101D3E0002ECF0A3EDF0D216AE27AF28900002E031
:101D4E00FCA3E0FDEFC39DEE9C40159000BAE0B4FD
:101D5E000104D2968002D295C21674C890002CF05F
:101D6E00A216B3B3500790002CE0B5370280159041
:101D7E0000BAE0B40104D2968002D29574C89000E5
:101D8E002CF0C21690002DE0B537028003021E35EE
:101D9E00A217406B900008E0FEA3E0FFEF4E605DDF
:101DAE00AC25AD26740ABC0033D39D402FAA29ABB7
:101DBE002A74058A048B05FF1200858D068C079008
:101DCE000008E0FCA3E0FDCFCECF12000374011299
:101DDE004C1D900008EEF0A3EFF08021AE29AF2A43
:101DEE00900008E0FCA3E0FD120003740A8E048F3D
:101DFE0005FF120085900008ECF0A3EDF0D217AEAF
:101E0E0027AF28900008E0FCA3E0FDEFC39DEE9CF9
:101E1E0040159000BAE0B40104C2968002C29574D7
:101E2E004690002DF0C217A217B3B3500790002DA5
:101E3E00E0B5370280159000BAE0B40104C2968076
:101E4E0002C295744690002DF0C217E54CB40C02F8
:101E5E008003021F4C90002FE0C394465013900055
:101E6E00BAE0B40104C2968002C2A0744690002F5C
:101E7E00F0855A34753300900032E0F55012009E12
:101E8E00E53690002FF090000AE533F0A3E534F02C
:101E9E00C219900065E02402FE90002FE0C39E5010
:101EAE0014900065E02402FE90002FE0F4042E90C2
:101EBE00002FF08012900065E02405FE90002FE0C8
:101ECE00F4042E90002FF09007A0E0F533A3E0F578
:101EDE0034900032E0F55012009EE53690002EF060
:101EEE00900004E533F0A3E534F0C218900065E0ED
:101EFE002402FE90002EE0C39E5014900065E02454
:101F0E0002FE90002EE0F4042E90002EF08012902F
:101F1E000065E02405FE90002EE0F4042E90002EC5
:101F2E00F0E549B4011574C890002AF074C8900009
:101F3E002CF074C890002EF0754900754C0390007B
:101F4E002EE0B537028003021FEFA218406B9000FF
:101F5E0004E0FEA3E0FFEF4E605DAC25AD26740AF3
:101F6E00BC0033D39D402FAA29AB2A74058A048B5B
:101F7E0005FF1200858D068C07900004E0FCA3E09F
:101F8E00FDCFCECF1200037401124C1D900004EE53
:101F9E00F0A3EFF08021AE29AF2A900004E0FCA35D
:101FAE00E0FD120003740A8E048F05FF1200859067
:101FBE000004ECF0A3EDF0D218AE27AF2890000489
:101FCE00E0FCA3E0FDEFC39DEE9C40159000BAE04F
:101FDE00B40104D2968002D2A0C21874C890002E0A
:101FEE00F0A218B3B3500790002EE0B5370280155B
:101FFE009000BAE0B40104D2968002D2A074C890C8
:10200E00002EF0C21890002FE0B537028003022098
:10201E00B6A219406B90000AE0FEA3E0FFEF4E60FF
:10202E005DAC25AD26740ABC0033D39D402FAA2982
:10203E00AB2A74058A048B05FF1200858D068C076A
:10204E0090000AE0FCA3E0FDCFCECF120003740196
:10205E00124C1D90000AEEF0A3EFF08021AE29AFD6
:10206E002A90000AE0FCA3E0FD120003740A8E041D
:10207E008F05FF12008590000AECF0A3EDF0D21947
:10208E00AE27AF2890000AE0FCA3E0FDEFC39DEE63
:10209E009C40159000BAE0B40104C2968002C2A022
:1020AE00744690002FF0C219A219B3B350079000D6
:1020BE002FE0B5370280159000BAE0B40104C29645
:1020CE008002C2A0744690002FF0C219E54CB402F3
:1020DE00028003022192123FA71240BE900064E0DC
:1020EE002545F55A90079CE0FEA3E0FF7414124CB0
:1020FE002B90000EE0FCA3E0FD74068F02FF120091
:10210E00858D078C038E048A058B06124B2D900746
:10211E00A0EEF0A3EFF09000BAE0B401087450BE48
:10212E0000059F4002800D74509007A0F8E4F0E87F
:10213E00A3F0801B9007A0E0FEA3E0FF74F0BE00AA
:10214E00039F500B74F09007A0F8E4F0E8A3F09012
:10215E0007A0E0FEA3E0FFE55A2FFF50010E900707
:10216E00A0EEF0A3EFF090003CE0B40103754C0A32
:10217E0090003CE0B40203754C0B90003CE0B403BD
:10218E0003754C0CE54CB401259000D1E0902BBEAC
:10219E00F8282873123D458012123D45800D123DE0
:0B21AE00CF8008123E7B8003123E7BB6
:0F2BBE000221A20221A70221AC0221B10221B6FD
:1021B900754C029000BCE0B4020280030222D49064
:1021C900005FE0D3953F506490005FE0F404253F41
:1021D900FE9000BFE08E00F5F0E884FF7E008F508E
:1021E900EFC39410500CEF8550F0A4FDACF08D5066
:1021F90080037550FF90005FE0D39550400B90002D
:102209005FE0C39550F54D8003754D009000DAE00D
:10221900D3954D40069000DAE0F54D9000DBE0C320
:10222900954D50069000DBE0F54D807190005FE020
:10223900C3953FFE9000BFE08E00F5F0E884FF7E75
:10224900008F50EFC39410500CEF8550F0A4FDACF3
:10225900F08D5080037550FF855034753300900020
:102269005FE02534FFAE3350010E8E338F3474FF97
:10227900BE0009D39F400585344D8003754DFF90FD
:1022890000DAE0D3954D40069000DAE0F54D900074
:10229900DBE0C3954D50069000DBE0F54DA208B395
:1022A900B350099000C7E0D3954E5002800A7407D5
:1022B900900039F0C2A2801375A710E5CDC3954DE2
:1022C9004004C2A28002D2A275A700E54BC39409BB
:1022D9004003022929A2EDB35003022929C2EDE5E1
:1022E9004B60030223A790006DE070030223967EE2
:1022F900017F00E5BE124C2BE5BD2FFF50010E8E6C
:10230900338F3490006DE0B401187410124C2B9087
:102319000063E08E048F05FF120085ED900034F014
:10232900802CAE33AF347410124C2B900063E08EC6
:10233900048F05FF120085900034E02DFD50010C3B
:1023490074018C068D07124C1DEF900034F0E544A2
:1023590060089000C9E06402600280219000CBE02F
:10236900B4011A900034E075F0E7A4FFAEF0E5443B
:102379008E048F05FF120085ED900034F090009FC8
:10238900E064016006900034E0F538800375380098
:10239900900069E07005754B01800375BB18E54B2A
:1023A900B40102800302253F900069E07003022511
:1023B9002E7E017F00E5BE124C2BE5BD2FFF50019B
:1023C9000E8E338F349000AFE0B4010F7E0F7FFF84
:1023D900AC33AD34124C8A8E338F349000D4E0B4D0
:1023E9000245AE33AF34900024E0FCA3E0FDEDD309
:1023F9009FEC9E400A900024E533F0A3E534F0AE4B
:1024090033AF34900026E0FCA3E0FDEFD39DEE9CB2
:10241900400A900026E533F0A3E534F0AE33AF343B
:102429007404124C1D8F3A9000D4E0704CAE33AF57
:1024390034900024E0FCA3E0FDEFD39DEE9C40091D
:10244900124C8A8E338F348006753400753300AE92
:1024590033AF347410124C2B900060E08E048F055A
:10246900FF1200858C338D347400D39D74019C4018
:102479000585343A8003753AFF90009FE0B4010264
:10248900800302252CA208B3B3500E900073E0A874
:1024990025B80005D395265003022526900074E03F
:1024A90075F019A4FFAEF09000B7E08E048F05FF18
:1024B9001200859000B0E0853AF0A4FFAEF0746494
:1024C9008D028C038E048F05FF120085EA2DFDEB2A
:1024D9003CFC8C338D34E544600F9000C9E0B402B4
:1024E900089000CBE0640160028017AE33AF34740A
:1024F900E7124C2BE5448E048F05FF1200858C33BF
:102509008D34900034E0A833B8000AD395344005DF
:102519008534388006900034E0F538800690003420
:10252900E0F5388003753A0090006CE07005754B52
:1025390002800375BB19E54BB4020280030225FA38
:1025490090006CE070030225E9E537D3940140035C
:102559000225E7900022E0FEA3E0FFE53E124C824F
:10256900900022EEF0A3EFF07E017F00E5BE124C51
:102579002BE5BD2FFF50010E8E338F349000D9E02B
:102589007013740A124C2B74518E048F05FF1200BC
:10259900858D3E8019AE33AF34740A124C2B8F04EB
:1025A9008E057E017F95CDCCCD124B2D8F3EE53E1C
:1025B900D394644003753E64900022E0FEA3E0FFDB
:1025C900E53E2FFF50010E900022EEF0A3EFF090B0
:1025D9000070E0048E048F05FF1200858D3E800394
:1025E900753E329000BCE07005754B03800375BBE6
:1025F90013E54BB4035E9000BCE060477E017F00A9
:10260900E5BE124C2BE5BD2FFF50010E8E338F34E2
:102619007404124C1D8F3F9000BEE0853FF0A4FD6D
:10262900ACF07464FF1200858D3F9000BDE0853FDA
:10263900F0A4FFAEF074FF8E048F05FF1200858DA4
:102649004E8003753F0090006AE07005754B048069
:102659000375BB17E54BB4040280030226FB900007
:102669006AE0B4017C7E017F00E5BE124C2BE5BD1A
:102679002FFF50010E7404124C1D8E338F349000BD
:1026890037E06012900037E014904A3B93A833B8C2
:102699000006953440028006900037E014F090005F
:1026A90037E0C394775013900037E004904A3B9386
:1026B900A833B80005D3953450028006900037E05E
:1026C90004F0900037E0FE900090E08E0088F0A4BE
:1026D900FFAEF074648E048F05FF1200858D408073
:1026E9000375400090006BE07005754B058003751C
:1026F900BB16E54BB40502800302278E90006BE000
:10270900B4017C7E017F00E5BE124C2BE5BD2FFF95
:1027190050010E7404124C1D8E338F34900038E032
:102729006012900038E014904AB493A833B80006B8
:10273900953440028006900038E014F0900038E0AB
:10274900C394775013900038E004904AB493A833A7
:10275900B80005D3953450028006900038E004F0A3
:10276900900038E0FE900096E08E0088F0A4FFAE5D
:10277900F074648E048F05FF1200858D4180037506
:10278900410075BB1FE54BB406337E017F00E5BEF2
:10279900124C2BE5BD2FFF50010E8E338F34740977
:1027A900124C2B74E68E048F05FF1200858D439021
:1027B9000072E07005754B07800375BB15E54BB4D6
:1027C900070280030228D0900072E070030228BF3C
:1027D9007E017F00E5BE124C2BE5BD2FFF50010E97
:1027E9008E338F347404124C1D8F42900072E0B402
:1027F90001159000C6E08542F0A4FFAEF0740712FF
:102809004C1DEF9007A9F0900072E0B402159000FA
:10281900C6E08542F0A4FFAEF07407124C1DEF909C
:1028290007A8F0900072E0B4030280030228BD906B
:1028390000B3E0701CE542C3940A5002D201E5429C
:10284900D394644002C201900092E090005EF0804F
:1028590063900092E070349000C6E08542F0A4FFD6
:10286900AEF074FF8E048F05FF120085ED90005EB7
:10287900F0AE25AF26741EBE0006D39F4002D201DA
:10288900E53AD394E54002C2018029E542C3940A9E
:10289900500DAE25AF26741EBE0004D39F50028092
:1028A90002D201E53AD394E54002C201900092E0D8
:1028B90090005EF080037542009000C9E0700575D4
:1028C9004B08800375BB14E54BB408509000C9E070
:1028D90060397E017F00E5BE124C2BE5BD2FFF500C
:1028E900010E8E338F34EFD39421EE940E4005758B
:1028F90044FF8015AE33AF347410124C2B74E38E41
:10290900048F05FF1200858D4480037544009000F3
:102919006DE0600575BB1A800375BB18054BD2ECD9
:10292900AE27AF28EFD394A8EE94615003022BACE5
:10293900C20E7537469000AEE070057549028003F6
:10294900754903C293C294C291C292C287C290E5EB
:10295900B554EFF5B5E5B554DFF5B5C296C295C2E4
:10296900A0C297C2A2C2A1E5B5547FF5B5E5B55499
:10297900BFF5B5A21EB34008E5B54404F5B5800618
:10298900E5B554FBF5B5A210B3500EE53AD394332F
:102999004007E53AC394CC4003022A42E5B5440115
:1029A900F5B5740D90005CF0900068E075F064A4D2
:1029B900FFAEF08E358F367402BE000AD39F4006F3
:1029C90075360275350075A71085F95085FA517E5F
:1029D900017F00E551124C2BE5502FFF50010E8E5F
:1029E900338F34AC35AD36EF2DFDEE3CFC8C358D97
:1029F90036D293D294D291E536F5FBE535F5FCE56F
:102A090036F5E9E535F5EAE536F5EBE535F5EC902A
:102A190000ACE0B4031ED292D287D290E536F5ED30
:102A2900E535F5EEE536F5FDE535F5FEE536F5CEA8
:102A3900E535F5CF75A700D210E53AC3941A5002CF
:102A4900C21090000C74FFF0A374DCF090008FE0CA
:102A5900900012F8E4F0E8A3F0C214C216C2187488
:102A6900C890002AF074C890002CF074C890002E09
:102A7900F0C211C212C213752600752500753C00FB
:102A8900C208756C0090001AE4F0A3F0754C1E9012
:102A9900079EE0FEA3E0FF7403124C2B7401124C55
:102AA9001D90079CEEF0A3EFF0900081E060051205
:102AB90042F88002C204900084E060051243E88075
:102AC90002C206A204300501B35017A204B340089C
:102AD900E5B54408F5B58006E5B554F7F5B5A204A2
:102AE9009205A206300701B35017A206B34008E5C4
:102AF900B54402F5B58006E5B554FDF5B5A20692D3
:102B090007C203752C00752B00900014E4F0A3F0A4
:102B1900900070E075F032A4FFAEF0900022EEF064
:102B2900A3EFF0900010E4F0A3F0C21F9000287406
:102B390075F0A37430F090005DE0C3943C501975B2
:102B49008D32758B00753D0CE54BB4090990005D1C
:102B5900E004F0754B00803BE54BB40903754B006D
:102B6900752800752700758D00758B00753D0090DF
:102B7900005CE0C39414500890005CE004F0800607
:102B8900741490005CF090005CE0B41406E5B55450
:102B9900FEF5B5E543C394415009740E900039F030
:062BA900120291020A4530
:1049C3000000010001400160018001A001C001E07D
:1049D30002000300039603B603D603F404000500A4
:1049E30005180530054805600578059005A805C03C
:1049F300060006140628063C066E068C00FF013FDF
:104A0300015F017F019F01BF01DF01FF02FF0395EA
:104A130003B503D503F303FF04FF0517052F05476C
:104A2300055F0577058F05A705BF05FF0613062755
:104A3300063B066F068B06A9DAD8D7D5D4D2D0CFDA
:104A4300CDCBC9C7C6C4C2C0BEBCBAB8B5B3B1AF7B
:104A5300ADABA8A6A4A2A09D9B99969492908D8B92
:104A630089878482807E7C79777573716F6D6B69BA
:104A7300676563615F5D5B5957565452504F4D4BA9
:104A83004A4847454442413F3E3C3B3A3937363535
:104A9300343231302F2E2D2C2B2A29282726252559
:104AA3002423222121201F1E1E1D1C1C1B1A1A1920
:104AB30019EEECEBEAE9E8E7E5E4E3E1E0DEDDDB70
:104AC300D9D8D6D4D2D0CECCCAC8C6C3C1BFBCBA3B
:104AD300B7B5B2B0ADABA8A5A3A09D9B9895929096
:104AE3008D8A8785827F7D7A7775726F6D6A686537
:104AF30063615E5C5A575553514F4D4B494745438C
:104B030042403E3C3B393836353332312F2E2D2B44
:104B13002A292827262524232221201F1E1D1D1C68
:0A4B23001B1A1A1918181716161598
:102BCD00750B00750A00AE0AAF0BAC08AD09EDC36D
:102BDD009FEC9E401674FF12007575CF01780B7433
:102BED000126F6500418E436F650DB22900033E04F
:102BFD00B4AA1C900764E0B43C159007A4E0FEA3B2
:102C0D00E0FFEF4E6009741EBE0004D39F50030217
:102C1D002D2775360075350075F8099007A4E0FE6F
:102C2D00A3E0FF74076F4E6006740E6F4E7006744E
:102C3D003A900764F09007A4E0FEA3E0FF7408BE8D
:102C4D00001ED39F401A7E017F089007A4E0FCA3CD
:102C5D00E0FD1DBDFF011C1200038E338F34801F5C
:102C6D009007A4E0FEA3E0FF7408124C828F048E3F
:102C7D00057E017F08CDCCCD1200038E338F34AE8F
:102C8D0035AF36740CD39F74019E5003022D22A2D2
:102C9D00F9B3407EE5364535700375A382AE35AF89
:102CAD003674016F4E700375A300AE35AF367402E6
:102CBD006F4E700D9007A5E075F002A4FDACF08D80
:102CCD00A3AE35AF3674036F4E700375A300AE35EA
:102CDD00AF367403BE00039F5013AC33AD34ED2FEC
:102CED00FFEC3EFE900060124C52E0F5A3AE35AF06
:102CFD0036EFB40B09EEB401057414120075AE3540
:102D0D00AF36EFB40B07EEB4010375F80D7835123D
:102D1D004C92022C8C900033E4F022753600753500
:102D2D000075F8099007A4E0FEA3E0FF7408BE004B
:102D3D001ED39F401A7E017F089007A4E0FCA3E0FC
:102D4D00FD1DBDFF011C1200038E338F34801F90BB
:102D5D0007A4E0FEA3E0FF7408124C828F048E05D9
:102D6D007E017F08CDCCCD1200038E338F34AE356E
:102D7D00AF367411D39F74019E5003022E58A2F9E1
:102D8D00B35003022E55E5364535700375A3D2AE0B
:102D9D0035AF3674016F4E700375A300AE35AF3687
:102DAD0074026F4E700D9007A5E075F002A4FDAC96
:102DBD00F08DA3AE35AF3674036F4E700375A3005F
:102DCD00AE35AF3674046F4E700375A300AE35AFDC
:102DDD003674056F4E700375A300AE35AF367406AD
:102DED006F4E700375A300AE35AF3674076F4E701E
:102DFD000375A300AE35AF3674086F4E700375A31F
:102E0D0000AE35AF367408BE00039F5016AC33AD1F
:102E1D0034ED2FFFEC3EFE90005B124C52E5A3F01B
:102E2D0075A300AE35AF36EFB41009EEB4010574DD
:102E3D0014120075AE35AF36EFB41007EEB40103C2
:102E4D0075F80D7835124C92022D7B227536007572
:102E5D00350075F809AE35AF367417BE0004D39F33
:102E6D005003022F31A2F9B35003022F2EE5364540
:102E7D0035700375A3D2AE35AF3674016F4E700346
:102E8D0075A300AE35AF3674026F4E700D9007A569
:102E9D00E075F002A4FDACF08DA3AE35AF36740332
:102EAD006F4E700375A300AE35AF3674046F4E7060
:102EBD000375A300AE35AF3674056F4E700375A361
:102ECD0000AE35AF3674066F4E700375A300AE3588
:102EDD00AF3674076F4E700375A300AE35AF367401
:102EED00086F4E700375A300AE35AF367408BE0083
:102EFD00039F500C900045124C52E5A3F075A300B2
:102F0D00AE35AF3674166F4E70057414120075AE73
:102F1D0035AF3674166F4E700375F80D7835124C4B
:102F2D0092022E6222900033E0B4AB028003022F96
:102F3D00CC75360075350075F809AE35AF3674129F
:102F4D00BE007CD39F4078A2F9B34070E53645357D
:102F5D00700375A382AE35AF3674016F4E70037575
:102F6D00A300AE35AF3674026F4E700D9007A5E01D
:102F7D0075F002A4FDACF08DA3AE35AF3674036FC2
:102F8D004E700375A300AE35AF367403BE00039FBC
:102F9D00500990004A124C52E0F5A3AE35AF36748D
:102FAD00116F4E70057414120075AE35AF36741175
:102FBD006F4E700375F80D7835124C92022F472223
:102FCD0090003AE4F074649007A4F8E4F0E8A3F0FC
:102FDD00122E5974C89007A4F8E4F0E8A3F09000FD
:102FED0051E0B4371A90004EE0900045F090004F3C
:102FFD00E0900046F0900050E0900047F080469041
:10300D00003A7401F074659007A4F8E4F0E8A3F0B9
:10301D00122E5974C89007A4F8E4F0E8A3F09000BC
:10302D0051E0B4371A90004EE0900045F090004FFB
:10303D00E0900046F0900050E0900047F08006745C
:10304D000290003AF090003BE4F074669007A4F80B
:10305D00E4F0E8A3F0122E5974C89007A4F8E4F038
:10306D00E8A3F0900050E0B4371290004EE09000CD
:10307D003FF090004FE0900048F0807690003B7458
:10308D0001F074679007A4F8E4F0E8A3F0122E594C
:10309D0074C89007A4F8E4F0E8A3F0900050E0B4F1
:1030AD00371290004EE090003FF090004FE09000FE
:1030BD0048F0803E740290003BF074689007A4F8CD
:1030CD00E4F0E8A3F0122E5974C89007A4F8E4F0C8
:1030DD00E8A3F0900050E0B4371290004EE090005D
:1030ED003FF090004FE0900048F080067403900090
:1030FD003BF022E55D2534FFAE3350010E900064A8
:10310D00124C52E0F55EE55D2534FFAE3350010EF5
:10311D000FBF00010E900064124C52E0F55F856503
:10312D0061E55EB55F05855E5D8041E55FD3955ECA
:10313D00401DE55FC3955E8560F0A4FFAEF0E561CF
:10314D008E048F05FF120085ED255EF55D801DE572
:10315D005EC3955F8560F0A4FFAEF0E5618E048FD0
:10316D0005FF120085EDF404255EF55D22E55FD3C4
:10317D00955E401DE55FC3955E8560F0A4FFAEF0E2
:10318D00E5618E048F05FF120085ED255EF55D80EE
:10319D001DE55EC3955F8560F0A4FFAEF0E5618E21
:1031AD00048F05FF120085EDF404255EF55D22E523
:1031BD003875F00484FF7E008F5DE53875F004846A
:1031CD00ADF07C008D60756504753301753400E5D7
:1031DD005DC3943F500512310080069001A3E0F5C8
:1031ED005D855D53755200900036E075F020A4FFAB
:1031FD00AEF09000B5E08E048F05FF1200858D5D59
:10320D0090009DE0D3953850030232C29000C1E08A
:10321D00D395384010ED9001A4124C67E0F555752B
:10322D0054000232BF90008CE0D395384043E55DE9
:10323D009001A4124C67E0F55EE55D9001C4124C5F
:10324D0067E0F55F9000C1E0F4042538F56090006B
:10325D008CE0FE9000C1E0F4042EF561E55EB55FF3
:10326D0005855E5D800312317A855D55755400804C
:10327D0041E55D9001C4124C67E0F55EE55D90019E
:10328D00E4124C67E0F55F90008CE0F4042538F50E
:10329D006090009DE0FE90008CE0F4042EF561E559
:1032AD005EB55F05855E5D800312317A855D55756E
:1032BD0054000233699000C4E0D395385011E55D98
:1032CD00900224124C67E0F5557554000233699055
:1032DD00008DE0D395385043E55D900204124C67A4
:1032ED00E0F55EE55D900224124C67E0F55F90001D
:1032FD008DE0F4042538F5609000C4E0FE90008D5B
:10330D00E0F4042EF561E55EB55F05855E5D800335
:10331D0012317A855D557554008041E55D9001E46B
:10332D00124C67E0F55EE55D900204124C67E0F526
:10333D005F90009DE0F4042538F56090008DE0FE6F
:10334D0090009DE0F4042EF561E55EB55F05855EA8
:10335D005D800312317A855D55755400229000D53C
:10336D00E0F562756511753302753400AE25AF2633
:10337D00E56275F00FA4FDACF0EDD39FEC9E4021FE
:10338D00E5628E048F05FF120085ED75F010A4FF28
:10339D00AEF0E53875F01184FD7C00ED2FF56380FE
:1033AD000EE53875F01184FF7E00EF24F0F563858E
:1033BD00635DE53875F01184AFF07E008F601231DA
:1033CD0000855D64AE25AF269000D5E075F00FA4A5
:1033DD00FDACF0EDD39FEC9E402875330275341093
:1033ED0085635D12310085645E855D5FAE25AF2618
:1033FD00E5628E048F05FF124C468D608562611269
:10340D00317A855D5375520075556475540022905F
:10341D0000D5E0F562756511753302753400AE2582
:10342D00AF26E56275F00FA4FDACF0EDD39FEC9ED9
:10343D004021E5628E048F05FF120085ED75F010B9
:10344D00A4FFAEF0E53A75F01184FD7C00ED2FF58B
:10345D0063800EE53A75F01184FF7E00EF24F0F5E0
:10346D006385635DE53A75F01184AFF07E008F6082
:10347D00123100855D64AE25AF269000D5E075F064
:10348D000FA4FDACF0EDD39FEC9E40287533027573
:10349D00341085635D12310085645E855D5FAE25F8
:1034AD00AF26E5628E048F05FF124C468D60856256
:1034BD006112317A855D5375520090009FE0B4041E
:1034CD0053E53875F00484FF7E008F5DE53875F0A7
:1034DD000484ADF07C008D60756504753301753421
:1034ED0000E55DC3943F500512310080069001A3A5
:1034FD00E0F55DAE52AF53E55D124C2B74648E0456
:10350D008F05FF120085AE52AF53EF2DFDEE3CFC43
:10351D008C528D537555647554002290006AE0B439
:10352D000146E54075F00584FF7E008F5DE5407531
:10353D00F00584ADF07C008D6075650575330575FE
:10354D003400E55DC39417500512310080069005D7
:10355D007BE0F55DAE54AF55E55D2FFF50010E7468
:10356D0064124C828E548F5590006BE0B40146E589
:10357D004175F00584FF7E008F5DE54175F0058492
:10358D00ADF07C008D60756505753305753448E5C6
:10359D005DC39417500512310080069005C3E0F508
:1035AD005DAE54AF55E55D2FFF50010E7464124CA6
:1035BD00828E548F5590007AE0B40249E543C3944E
:1035CD004175F00584FF7E008F5DE54375F0058440
:1035DD00ADF07C008D60756505753306753400E5BD
:1035ED005DC3941350051231008006900677E0F507
:1035FD005DAE54AF55E55D2FFF50010E7464124C56
:10360D00828E548F559000BCE0B4020280030236C6
:10361D00C7E53875F01584FF7E008F5DE53875F0D0
:10362D001584ADF07C008D607565157533037534AB
:10363D00F4E55DC3940B50051231008006900463D0
:10364D00E0F55DE55D75F0FFA4FFAEF09000BDE027
:10365D008E048F05FF120085ED90005FF0E53F753C
:10366D00F078A4FFAEF074FF8E048F05FF12008575
:10367D008C338D3474028C068D07124C1D8F5DAC0E
:10368D0033AD347404FF124C468D6075650475338B
:10369D000675346EE55DC3941D500512310080062C
:1036AD009006EFE0F55DAE54AF55E55D2FFF50018F
:1036BD000E7464124C828E548F5522900072E0B4B9
:1036CD0001179007A9E02555FFAE5450010E90004B
:1036DD00C6E0124C828E548F55900072E0B40316E2
:1036ED00A201B3B3501090005EE0C39405A825B8B5
:1036FD000006952640028010900094E02555FFAEFF
:10370D005450010E8E548F5590006CE0B40202801F
:10371D00030238F590006FE0602FE540D3941E4012
:10372D0028900014E0FEA3E0FF9000AAE075F003DE
:10373D00A4FDACF0EFD39DEE9C400E9000CEE0A822
:10374D0025B80005D3952650030238F59000B7E053
:10375D008538F0A4FFAEF07405124C2B7407124C93
:10376D001D8E338F34900076E0A825B80004952681
:10377D005012900077E075F002A4FDACF0EFC39D00
:10378D00EE9C40030238F5E53875F00B84FF7E00A2
:10379D009005F4124C52FEE0FFEE90006EE0FEEF4D
:1037AD008E0088F0A4FFAEF074648E048F05FF12B6
:1037BD0000858C338D34900036E075F018A4FFAE83
:1037CD00F09000B5E08E048F05FF1200858C068DFC
:1037DD000790060C124C52AE33AF34E0124C2B74E2
:1037ED00648E048F05FF1200858C338D34E53EA861
:1037FD0033B80077D395344072E53EC39534FFE47A
:10380D009533FE8E338F347428BE00039F500C7594
:10381D003428753300740D900039F0AE33AF349009
:10382D00006FE0124C2B74288E048F05FF1200855B
:10383D008C338D34AE52AF53740A8E048F05FF1244
:10384D0000858D068C07AC33AD34CFCECF1200037F
:10385D00740A8E048F05FF1200858C338D34AE52A1
:10386D00AF53124C8A8E528F53807DE53EA833B8EC
:10387D00000495345072AE33AF34E53E124C828E57
:10388D00338F347428BE00039F500C753428753364
:10389D0000740D900039F0AE33AF3490006FE0122C
:1038AD004C2B74288E048F05FF1200858C338D34BC
:1038BD00AE52AF53740A8E048F05FF1200858D062C
:1038CD008C07AC33AD34CFCECF120003740A8E0407
:1038DD008F05FF1200858C338D34AE52AF53EF2D13
:1038ED00FDEE3CFC8C528D5322AE52AF53AC54AD19
:1038FD005512000374648E048F05FF1200858C52DF
:10390D008D53900067E08C068D07124C2B74648EDE
:10391D00048F05FF1200858C528D53A2084017AEFF
:10392D0025AF267405BE00039F5002D208E53AD399
:10393D0094CC4002D2029000C9E0B402089000CBB2
:10394D00E0640160028017AE52AF53E544124C2B78
:10395D0074E78E048F05FF1200858C528D539000F5
:10396D0089E05402601B900080E0A825B80012D3B6
:10397D009526400DA208B3B35007E53AC3949A407B
:10398D00028028AE5BAF5C90007EE075F002A4FD76
:10399D00ACF0EF2DFDEE3CFC74022DFD50010CE55D
:1039AD003ABC0007D39D4003756901853A5C755B90
:1039BD0000E5697003023A4C9000DCE0C395694064
:1039CD0070E54075F00584FF7E00900564124C5241
:1039DD00E0F534753300AE33AF3490008EE0124C09
:1039ED002B74648E048F05FF1200858C358D3690F7
:1039FD0000DCE004C395698C068D07124C2B9000FA
:103A0D00DCE08E048F05FF1200858C358D3690001D
:103A1D007FE08C068D07124C2B740A8E048F05FFE8
:103A2D00120085AE52AF53EF2DFDEE3CFC8C528D46
:103A3D005305699000DCE0C39569500375690090EA
:103A4D000089E05401601B90007DE0A825B80012AC
:103A5D00D39526400DA208B3B35007E538C394CCD7
:103A6D004002802590007BE075F003A4FFAEF0E5E9
:103A7D00662FFF50010E74032FFF50010EE538BE67
:103A8D000007D39F4003756A01853866E56A7003A8
:103A9D00023B279000DDE0C3956A4070E54075F06C
:103AAD000584FF7E00900564124C52E0F5347533A9
:103ABD0000AE33AF3490008EE0124C2B74648E0444
:103ACD008F05FF1200858C358D369000DDE004C327
:103ADD00956A8C068D07124C2B9000DDE08E048FBD
:103AED0005FF1200858C358D3690007CE08C068D9F
:103AFD0007124C2B740A8E048F05FF120085AE52EF
:103B0D00AF53EF2DFDEE3CFC8C528D53056A9000AA
:103B1D00DDE0C3956A5003756A0090008EE0A852EF
:103B2D00B800049553500990008EE0F5537552007E
:103B3D00229000CAE0B401028003023C49A208B3FE
:103B4D005003023C47900095E0B40168AE52AF536C
:103B5D00AC25AD26120003743C8E048F05FF1200B8
:103B6D00859000A5E0BC00109D400D9000A7E0A839
:103B7D0052B8000495535002D203AE52AF53AC2548
:103B8D00AD26120003743C8E048F05FF1200859044
:103B9D0000A5E0C3940ABC0015D39D40119000A769
:103BAD00E0C39405A852B80005D395535002800286
:103BBD00C2038068AE52AF53AC25AD26120003741C
:103BCD00788E048F05FF1200859000A5E0BC0010D3
:103BDD009D400D9000A7E0A852B8000495535004E5
:103BED00D2038038AE52AF53AC25AD26120003740C
:103BFD00788E048F05FF1200859000A5E0C3940A0E
:103C0D00BC0015D39D40119000A7E0C39405A852A8
:103C1D00B80005D3955350028002C203A203B340EE
:103C2D0019AE52AF539000A6E0124C2B74648E0463
:103C3D008F05FF1200858C528D538002C2039000B8
:103C4D00CAE0B40258E53875F00884FF7E008F5D38
:103C5D00E53875F00884ADF07C008D6075650875EC
:103C6D0033017534E0E55DC3943F5005123100809A
:103C7D0006900263E0F55DE55D75F05EA4FFAEF0C4
:103C8D00740A8E048F05FF1200858C568D577402B1
:103C9D00BC000AD39D4006755702755600A200B3AD
:103CAD004006A202B3B3500990001AE4F0A3F080CD
:103CBD0024AE52AF537400D39F74019E400C9000FC
:103CCD001AE552F0A3E553F0800B74FF90001AF83B
:103CDD00E4F0E8A3F09000ACE0D394024006A20813
:103CED00B3B34002800DAE52AF537402124C2B8E03
:103CFD00528F53900095E0B4010DAE52AF53740244
:103D0D00124C2B8E528F53AE52AF53745E124C2BFE
:103D1D00740A8E048F05FF1200858C528D53740228
:103D2D00BC000AD39D4006755302755200900018D1
:103D3D00E552F0A3E553F022900036E090036412B3
:103D4D004C67E0F567756864900036E0FE9000A062
:103D5D00E0D39E4037E53875F00884FF7E008F5D17
:103D6D00E53875F00884ADF07C008D6075650875DB
:103D7D003303753496E55DC3941F500512310080F1
:103D8D0006900419E0F55D855D688035E53875F0C0
:103D9D000884FF7E008F5DE53875F00884ADF07CFA
:103DAD00008D607565087533037534B6E55DC39494
:103DBD001F50051231008006900439E0F55D855DD8
:103DCD0068229000D6E0F56275651175330475347F
:103DDD0000AE25AF26E56275F00FA4FDACF0EDD376
:103DED009FEC9E4021E5628E048F05FF120085ED4C
:103DFD0075F010A4FFAEF0E53875F01184FD7C0070
:103E0D00ED2FF563800EE53875F01184FF7E00EF20
:103E1D0024F0F56385635DE53875F01184AFF07EB0
:103E2D00008F60123100855D64AE25AF269000D6FF
:103E3D00E075F00FA4FDACF0EDD39FEC9E4028751E
:103E4D00330475341085635D12310085645E855DC4
:103E5D005FAE25AF26E5628E048F05FF124C468DB1
:103E6D006085626112317A855D67756864229000A4
:103E7D00D6E0F562756511753304753400AE25AF66
:103E8D0026E56275F00FA4FDACF0EDD39FEC9E40DE
:103E9D0021E5628E048F05FF120085ED75F010A4EB
:103EAD00FFAEF0E53A75F01184FD7C00ED2FF56362
:103EBD00800EE53A75F01184FF7E00EF24F0F56376
:103ECD0085635DE53A75F01184AFF07E008F601269
:103EDD003100855D64AE25AF269000D6E075F00FFC
:103EED00A4FDACF0EDD39FEC9E40287533047534E2
:103EFD001085635D12310085645E855D5FAE25AF13
:103F0D0026E5628E048F05FF124C468D6085626139
:103F1D0012317A855D677568649000D1E0B40479DB
:103F2D00900036E0FE9000A0E0D39E4037E5387556
:103F3D00F00884FF7E008F5DE53875F00884ADF0E4
:103F4D007C008D60756508753303753496E55DC32A
:103F5D00941F50051231008006900419E0F55D851F
:103F6D005D688035E53875F00884FF7E008F5DE56E
:103F7D003875F00884ADF07C008D6075650875337B
:103F8D00037534B6E55DC3941F50051231008006EC
:103F9D00900439E0F55D855D682290006AE0B4011A
:103FAD003BE54075F00584FF7E008F5DE54075F0C3
:103FBD000584ADF07C008D60756505753305753430
:103FCD0018E55DC3941750051231008006900593D6
:103FDD00E0F55DE568255DC39464F56890006BE0E0
:103FED00B4013BE54175F00584FF7E008F5DE54131
:103FFD0075F00584ADF07C008D6075650575330534
:10400D00753460E55DC3941750051231008006903C
:10401D0005DBE0F55DE568255DC39464F568E5674E
:10402D002568F55A900072E0B402109007A8E025BB
:10403D005AFE9000C6E0F4042EF55A9000C9E0D364
:10404D0094014040E544C394E7501D74E7C3954483
:10405D00FE9007AAE08E00F5F0E884FF7E008F5DEC
:10406D00E55A255DF55A801CE544C394E7FE90079B
:10407D00AAE08E00F5F0E884FF7E008F5DE55AC35F
:10408D00955DF55AA2084006E5672464F55AE55A90
:10409D00D394644009E55AC39464F55A8003755A64
:1040AD00009000A2E0C3955A50069000A2E0F55A88
:1040BD0022D2009000B8E0A825B800049526503B08
:1040CD009000B8E0A825B8000495265003755A0F46
:1040DD009000B8E004A825B8000495265003755A41
:1040ED000A9000B8E02402A825B8000495265005D2
:1040FD00755A05C2007409900039F07E017F009059
:10410D0000A8E0124C2B9000B7E08E048F05FF1233
:10411D000085E538BC000CD39D4008C200740A90A0
:10412D000039F09000A9E0C39540500D9000BBE020
:10413D00A825B80006952640028008C200740B9091
:10414D000039F0A2004003755A05900072E0B403E7
:10415D0006A201B3B34002802B90005EE0C394052C
:10416D00A825B800049526500C900093E0F55A74DC
:10417D000C900039F090005EE0A825B8000495265B
:10418D005002C200855A45900064E0255AFE900009
:10419D0036E075F01E84FC7F00EE2CF55A2290005F
:1041AD0036E075F00584FF7E008F5D900036E0757A
:1041BD00F00584ADF07C008D607565057533037574
:1041CD0034D69000B5E01475F00584FF7E00E55DF2
:1041DD00BE00039F5005123100800BE55D90043A3F
:1041ED00124C67E0F55DE55D9007ABF09007ABE035
:1041FD00FE9000A4E0C39E50089000A4E09007AB91
:10420D00F022E54075F00584FF7E00900564124CA8
:10421D0052E0F56CE56CD394644010E56CC3946486
:10422D0075F00F84FF7E008F6C8003756C0090001D
:10423D0087E0256CF56C2290079EE0FEA3E0FF74ED
:10424D0004124C1DE538124C2B740F8E048F05FF94
:10425D0012008590079CECF0A3EDF090007AE0B48D
:10426D000262E543C3944175F00584FF7E008F5DC6
:10427D00E54375F00584ADF07C008D6075650575C1
:10428D003306753414E55DC3941750051231008063
:10429D000690068BE0F55D90079CE0FEA3E0FF74B1
:1042AD000A8E048F05FF120085E55D8C068D0712C1
:1042BD004C2B740A8E048F05FF12008590079CEC21
:1042CD00F0A3EDF090079CE0FEA3E0FF9007A2E0C5
:1042DD00FCA3E0FDEDD39FEC9E400F9007A2E0F80C
:1042ED00A3E090079CC8F0A3C8F022900081E0B431
:1042FD000103852650900081E0B402129000B7E0D2
:10430D008538F0A4FFAEF07408124C1D8F5090004C
:10431D0081E0B40303853A50900081E0B404038535
:10432D004050900081E0B40507E541C39414F55069
:10433D00900081E0B40603854250900081E0B407FF
:10434D0003854350900081E0B408038544509000EC
:10435D0081E0B40903853F50900082E0FE90008318
:10436D00E0D39E404B900081E0B40418900083E0B0
:10437D00C395505002D204900082E0D39550400274
:10438D00C204802A900082E0C395505009900083AA
:10439D00E0D3955050028002D204900082E0D39574
:1043AD00505009900083E0C395505002C204802AFA
:1043BD00900082E0D395504009900083E0C3955062
:1043CD0040028002C204900082E0C39550400990E3
:1043DD000083E0D395504002D20422900084E0B4D3
:1043ED000103852650900084E0B402129000B7E0DE
:1043FD008538F0A4FFAEF07408124C1D8F5090005C
:10440D0084E0B40303853A50900084E0B40403853E
:10441D004050900084E0B40507E541C39414F55075
:10442D00900084E0B40603854250900084E0B40708
:10443D0003854350900084E0B408038544509000F8
:10444D0084E0B40903853F50900085E0FE9000861E
:10445D00E0D39E4040900085E0C3955050099000F8
:10446D0086E0D3955050028002D206900085E0D3AD
:10447D0095505009900086E0C395505002C20690A9
:10448D000084E0B401099000C3E0D3953A50028056
:10449D0002C206802A900085E0D395504009900015
:1044AD0086E0C3955040028002C206900085E0C3AD
:1044BD0095504009900086E0D395504002D20622D7
:1044CD00AE58AF5974F5D39F74019E4008785812B9
:1044DD004C920245C8755901755800AE25AF26E5B9
:1044ED006CBE000DD39F4009900099E0D3956D40AF
:1044FD0002801B756D00E56CC39526F55090009CF0
:10450D00E0D3956B4006E56B2550F56B8002056D8C
:10451D00900075E0D3953A401CE538C395394015A8
:10452D00AE25AF26E56CBE00039F500990009AE0C2
:10453D00D3956E400280579007ACE0A825B80004D3
:10454D00952650037570009007ACE0A825B8000BB8
:10455D00D395264006E5269007ACF0E570702AE568
:10456D0026C3956CF550E550D39405400375500561
:10457D0090009BE0C3956B5007E550C3956B4002CF
:10458D008007E56BC39550F56B756E008002056E67
:10459D00E5707016900075E0C3953A500DE56C24EA
:1045AD0005A825B8000695264002800F900088E0EA
:1045BD00F56B75700174789007ACF022AE58AF5959
:1045CD0074E9D39F74039E40087858124C920247A9
:1045DD0076755901755800756B32A220402A756B9E
:1045ED0019900088E075F002A4FFAEF0E56DBE00F5
:1045FD0006D39F4002D220056D7570037478900725
:10460D00ACF0756F00024765AE25AF26E56C6F4EB9
:10461D007003024765E56CBE000DD39F4009900005
:10462D0099E0D3956D40028017756D00A208B3B364
:10463D005007E570C3940340028003756B19800D1C
:10464D00E56CC39526F550E56D2550F56D9000751B
:10465D00E0D3953A400E9007ACE0A825B80007D3FB
:10466D0095264002800C056F900088E0B56F0375AC
:10467D007000E570B4030DE56C2402A825B80006A2
:10468D0095264002800A056FE56FB43C03757002F4
:10469D00E570B402299007ACE0A825B8000ED395BB
:1046AD00264009E5269007ACF0756F00900075E087
:1046BD00C3953A5009756F0074789007ACF0E570AA
:1046CD00705A900075E0D3953A401CE538D3953972
:1046DD004015AE25AF26E56CBE00039F5009900036
:1046ED009AE0D3956E40028008756E00756B4B8015
:1046FD0028E526C3956CF550E550D3940540037518
:10470D005005900075E0D3953A4008E56E2550F5BB
:10471D006E8006E56E2406F56E756F00E5707016F9
:10472D00900075E0C3953A500DE56C2405A825B8A9
:10473D000006952640028003757001E570B40118DE
:10474D00756B19056F900088E0B56F067570027571
:10475D006F0074789007ACF0E56B75F00AA4FFAEAE
:0A476D00F09007A6EEF0A3EFF02293
:094C67002582F58250020583222A
:0F4C0E0025E050020583258250020583F582229E
:10006400EF2F500205832582F582E5833E2EF5832A
:010074002269
:104C8200CFC39FFF50011E22C3EF9DFFEE9CFE2269
:094C7000E493F608740193F622A6
:084C92000806B6000218062214
:0D4C3900A3E004F07006124C5DE004F022D0
:0E003900A3E014F0B4FF06124C5DE014F022B8
:0E4C1D00048007C3CE13CECF13CFD5E0F6220E
:104B2D00BC000FBE0008ED8FF084FFADF022E4FE57
:104B3D00FF22BE000DEF60FE54F0606F20E7030210
:104B4D004BE3EAC0E0EBC0E078017A0075F001EECE
:104B5D0020E710EF25E0FFEE33FE0AC5F023C5F088
:104B6D0030E7F0EA5407F9096A7A007B0060010822
:104B7D00C3EC9E40167004ED9F4010ED9FFDEC9E22
:104B8D00FCE5F0CA4ACA03F5F08005E5F003F5F03F
:104B9D00C3EE13FEEF13FFD9D77908CACBCAD8D00D
:104BAD00EAFEEBFFD0E0FBD0E0FA22EC8FF084FCC4
:104BBD00ED54F045F0C48FF084FEEDC454F045F093
:104BCD00C48FF084FDEEC4FE54F02DFFEE540F3C67
:104BDD00FEADF07C0022790078008FF0EC7E08208D
:104BED00E70DC3CD33CD33C933C9C833C8DEF08427
:104BFD0049F9E5F08FF0BE00E6FD7C00E9FFE8FE27
:014C0D002284
:0E4C2B00F88FF0A4FFE5F0CE88F0A42EFE2254
:10000300EF8DF0A4F9A8F0EF8CF0A428F8EE8DF0B2
:06001300A428FEE9FF2213
:10007500600D782B02007F007830D8FED5E0F8229D
:10008500EEC0E07E00124B2DEFFDEEFCD0E0FE222F
:0C4C4600EEC0E07E00124B2DD0E0FE22FC
:03001B0002001EC2
:03009B0002004917
:03000000024C7936
:094C790075817175D0000203B9C8
:104C5200E5822FF582E5833EF583220582D5820225
:054C62001583158222FC
:10001E00C0E0C0F0C083C082C0D075D00012035BB8
:0B002E00D0D0D082D083D0F0D0E032E0
:10004900C0E0C0F0C083C082C0D075D00012035E8A
:0B005900D0D0D082D083D0F0D0E032B5
:00000001FF
